:020000040000FA
:04000000FA3060284A
:080008008612601C8616AE0092
:10001000030EAF008312051E13284008E000601C89
:10002000861660188612051D1728BC0B1328283069
:10003000BC000F30A3008B100314851E0310E00CCE
:0A0040002F0E8300AE0E2E0E0900F5
:1000C000203084008001840A80300402031C6228EE
:1000D0002830BC008316FF3085055F3086055F3011
:1000E00087058312850186018701103083168E00F3
:1000F0008312703083168F0083120030031799002B
:100100000313003003179A000313003097000030E8
:100110009F00003083169F008312003003179E005B
:100120000313003003179F000313C73083168100A9
:10013000831230309000003092000030831694001B
:10014000831200309400A63083169800831200308A
:1001500083169B0083120030980033308316990079
:100160008312003083168C008312003083168D00BA
:10017000831210308B00B20BBB280130A400810128
:100180008E018F010B118B100B108C128C018D01C5
:100190008B1764000B19D720E620C92848085002A5
:1001A000031DD4285008C0004808D00008000B11D7
:1001B000A40B08000430A400A3080319E228861346
:1001C000A303080006098039860008000608A0007D
:1001D0000708A1002118F1280130A5070318F62807
:1001E000FD280130A502031CFA28FD28FF30A500D8
:1001F0004814FD28A5014810FD28A1180429013044
:10020000A6070318092910290130A602031C0D298D
:100210001029FF30A600C8141029A601C810102903
:10022000211917290130A70703181C292329013098
:10023000A702031C20292329FF30A70048152329E2
:10024000A70148112329201A2A290130A8070318D9
:100250002F2936290130A802031C33293629FF3003
:10026000A800C8153629A801C8113629211A3D2928
:100270000130AA070318422949290130AA02031CA8
:1002800046294929FF30AA0048164929AA014812DF
:100290004929201B50290130AB07031855295C2937
:1002A0000130AB02031C59295C29FF30AB00C81692
:1002B0005C29AB01C8125C29211B63290130AC0702
:1002C000031868296F290130AC02031C6C296F29BF
:1002D000FF30AC0048176F29AC0148136F29A119F2
:1002E00076290130AD0703187B2982290130AD0240
:1002F000031C7F298229FF30AD00C8178229AD0178
:10030000C8138229CE2008000708803A8700080019
:100310000708203A870008000608803A860008008F
:084000000800000000000700A9
:02400E00CC03E1
:00000001FF
